:1000000012C02CC02BC02AC029C028C027C026C0BF
:1000100025C024C023C022C021C020C01FC01EC0D4
:100020001DC01CC01BC011241FBECFE5D4E0DEBF25
:10003000CDBF10E0A0E6B0E0E4ECF2E002C0059035
:100040000D92A036B107D9F710E0A0E6B0E001C0EC
:100050001D92A036B107E1F7F8D033C1D1CFCF93CD
:10006000DF93CDB7DEB7E8E3F0E01082E5E3F0E040
:1000700080E28083E2E3F0E01082E7E3F0E01082C8
:10008000E4E3F0E080E28083E1E3F0E01082DF91DE
:10009000CF910895CF93DF93CDB7DEB726970FB6F4
:1000A000F894DEBF0FBECDBF6B837C838D839E83B0
:1000B0008B819C81AD81BE81880F991FAA1FBB1FB8
:1000C000880F991FAA1FBB1F880F991FAA1FBB1F4C
:1000D000880F991FAA1FBB1F9C01AD0180E092E110
:1000E000AAE7B0E0BC01CD01CAD0DA01C90101978D
:1000F0009A838983E0E4F0E089819A81892F990FBE
:10010000990B8083E9E2F0E089818083EAE2F0E004
:1001100088E18083E0E4F0E086E8808326960FB6ED
:10012000F894DEBF0FBECDBFDF91CF910895CF937E
:10013000DF93CDB7DEB722970FB6F894DEBF0FBEC0
:10014000CDBFEBE2F0E08081882344F4ECE2F0E004
:100150008081282F33273A83298302C01A8219828B
:1001600089819A8122960FB6F894DEBF0FBECDBF6B
:10017000DF91CF910895CF93DF93CDB7DEB721976D
:100180000FB6F894DEBF0FBECDBF8983EBE2F0E07F
:1001900080819927807290700097C1F3ECE2F0E0C3
:1001A0008981808321960FB6F894DEBF0FBECDBF44
:1001B000DF91CF910895CF93DF93CDB7DEB723972B
:1001C0000FB6F894DEBF0FBECDBF89838981282F7B
:1001D00033273B832A838A819B81009731F02A81D0
:1001E0003B812130310549F010C0A5E3B0E0E5E3E3
:1001F000F0E080818F7D8C931FC0A5E3B0E0E5E344
:10020000F0E0808180628C9317C0E5E3F0E08081AC
:10021000992780729070009741F0A5E3B0E0E5E384
:10022000F0E080818F7D8C9307C0A5E3B0E0E5E32B
:10023000F0E0808180628C9323960FB6F894DEBF45
:100240000FBECDBFDF91CF910895CF93DF93CDB790
:10025000DEB721970FB6F894DEBF0FBECDBFFFDE2D
:1002600060E875E280E090E015DF00C060DF898320
:1002700089818823D9F389818F5F7DDFF7CFA1E260
:100280001A2EAA1BBB1BFD010DC0AA1FBB1FEE1F10
:10029000FF1FA217B307E407F50720F0A21BB30B5B
:1002A000E40BF50B661F771F881F991F1A9469F7D7
:1002B00060957095809590959B01AC01BD01CF0133
:0402C0000895FFCFCF
:00000001FF
